:020000040000FA
:100000002E288207003400340034003400341B34BE
:1000100077344034003435346734E03400346A34A3
:10002000CF34C03400349A341D3420340034D534F5
:100030009F34803401341334B234203401344034DA
:100040006F34403401347B34CA3490340134AB34DF
:100050003F3400340134C934C33480348B018316F7
:100060008113FB308500860183120511B220D22056
:10007000051A3B28AB21890119230808A30019237D
:100080000808A40019230808A50019230808A600D9
:10009000192308088C00192308088D001923080863
:1000A0008E00192308088F006F229D221E225522E0
:1000B00055220508B30003303305B200B0014030CB
:1000C000AF00B401B7014921B3196828882063281B
:1000D0009D019C019B0101309A00331A7928E83078
:1000E0009A0003309B00792803109A0D9B0D9C0DFC
:1000F0009D0DAF0DB00D031C7428B4188128362156
:100100008328F92011216F229D221E225522632867
:10011000B41894280430B702D7303707031C92284C
:100120002830B700A0209B280430B707D730370706
:100130000318B701A0206F229D221E22552208001D
:10014000370801208F00B70A370801208E00B70A50
:10015000370801208D00B70A370801208C000330D2
:10016000B702080029230330860006162923061249
:100170000330860006162C2306120330860006166E
:100180002C2306120230860006162F230612283072
:10019000EA220830EA220130EA220630EA220C3054
:1001A000EA2208008030EA225030EE224930EE2266
:1001B0004330EE224530EE224C30EE226730EE2204
:1001C0006530EE226E30EE22C030AB00EA222030E5
:1001D000EE227630EE223530EE222E30EE22313015
:1001E000EE222D30EE223330EE223030EE221E236E
:1001F00008001A088C07031C02298D0F02298E0F94
:1002000002298F0A1B088D07031C09298E0F092953
:100210008F0A1C088E07031C0E298F0A1D088F07E2
:100220000800FE300F0703182D2901300F02031CB0
:10023000352936300E0703182D29C9300E02031C4C
:1002400035293C300D0703182D29C3300D02031C3E
:10025000352980300C02031C352980308C00C330D6
:100260008D00C9308E0001308F0008009A099B096B
:100270009C099D099A0F41299B0F41299C0F4129F7
:100280009D0AF9208F1F48298C018D018E018F0155
:100290000800B0014030AF007221B01B5329083074
:1002A000AF070318B00A0508B30003303305B100E7
:1002B000320603194C290310B20D3108B206320878
:1002C0000239B500340603196A293508B40031082B
:1002D000B2004C29B401B21C6F290230B4003108BD
:1002E000B2000800051E7729851980297C29851907
:1002F0007E293918822995293914AA293910AA2961
:10030000B901AA291030BA00051A8B292623BA0B85
:1003100084290F22AA299D010F309C0042309B00A6
:1003200040309A00F9201121A6291030BA00851911
:100330009E292623BA0B97290F22AA299D010F3047
:100340009C0042309B0040309A0036216F229D2253
:100350001E225522080080308C0096308D00983087
:100360008E0000308F00890119230808A30019238B
:100370000808A40019230808A50019230808A600E6
:100380006F229D22C430AB00EA224330AB00EE2244
:100390004130AB00EE224C30AB00EE221E22552243
:1003A00049219D019C019B0110309A003319DA29E3
:1003B00080309A000000B418E8299A099B099C092A
:1003C0009D099A0FE8299B0FE8299C0FE8299D0AAF
:1003D0001A08A307031CF129A40FF129A50FF1297D
:1003E000A60A1B08A407031CF829A50FF829A60ACA
:1003F0001C08A507031CFD29A60A1D08A607051E43
:10040000CE298901230888000C23240888000C23A6
:10041000250888000C23260888000C2308000430D7
:1004200089000C0888000C230D0888000C230E0896
:1004300088000C230F0888000C2308009501960102
:100440009701980199012030A0002308A7002408F3
:10045000A8002508A9002608AA000310271C472A7F
:100460000C089607031C392A970F392A980F392A46
:10047000990A0D089707031C402A980F402A990AE9
:100480000E089807031C452A990A0F089907990C2A
:10049000980C970C960C950CAA0CA90CA80CA70C00
:1004A000A00B2D2A003099000800153084000008A8
:1004B000A2000830A100A20C031C622A86150615B2
:1004C0000611652A861106150611A10B5B2A840AFE
:1004D0001A300402031C572A86178613080020309E
:1004E0009E009001910192019301940103108C0DE3
:1004F0008D0D8E0D8F0D03180C14900D910D920D16
:10050000930D940D9E03031D862A0800103084006D
:100510009222840A9222840A9222840A9222840AD3
:100520009222762A033000079F009F198000303006
:1005300000079F009F1B800008008030EA222030C7
:10054000EE22130E0F39303EEE2213080F39303EE3
:10055000EE222C30EE22120E0F39303EEE2212081F
:100560000F39303EEE22110E0F39303EEE222E3082
:10057000EE22C030EA2211080F39303EEE22100E72
:100580000F39303EEE2210080F39303EEE22203077
:10059000EE226B30EE224830EE227A30EE2220300E
:1005A000EE220800860183160830860083120613A7
:1005B0008616FF30AD0006160608AC0006120000D5
:1005C0000000061600000612AD030319E92AAC1953
:1005D000DB2A0800AB00B8010613F12AAB0038147F
:1005E0000617D222860183160030860083128612F7
:1005F000061338180617F03086052B0E0F398604BF
:10060000061600000612F03086052B080F39860406
:1006100006160000061208008316081555308900DA
:10062000AA30890088148818132B08118312890AAC
:100630000800831608148312890A08002323232341
:10064000232323230800262326230800FF30AD00A0
:10065000342B8030AD00342B4030AD00342B2030B3
:10066000AD00342B1030AD00FF30AE00AE0B362B9A
:06067000AD0B342B080065
:084000007F007F007F007F00BC
:02400E00F13F80
:10420000C4001D00F3002A0028000100D6000000B1
:10421000000000000000000000000000000000009E
:10422000000000000000000000000000000000008E
:10423000000000000000000000000000000000007E
:10424000000000000000000000000000000000006E
:10425000000000000000000000000000000000005E
:10426000000000000000000000000000000000004E
:10427000000000000000000000000000000000003E
:00000001FF
